:100000000428FF3FFF3FFF3F83160030850010307C
:10001000860083120610861006116220323090008E
:100020009E20900B10283F308B2000308B206620C4
:1000300006149E2086149E2086109E2006106620A0
:100040007A207A201108AE00AD00443091060319E1
:1000500037282230AD0603194B287A207A207A20DF
:1000600062209E206F308B2000308B201F287A204A
:100070007A207A2062205030061AA030AF00861411
:100080009E2086100530061A0A30AF0790308B206C
:100090002F088B201F287A207A207A2062209E2029
:1000A00090308B2022308B209E2006149E2006103C
:1000B0009E208614643090009E20900B5C28861051
:1000C0009E201F288316051283120800831605162A
:1000D000831208008D008D0908308E0005129E20C5
:1000E00003108D0D03180516031C05129C208E0BA2
:1000F000702808009101051A99289720083090006F
:100100000310910D051A11149E20900B8028972042
:10011000910908009E206A2005169E2005169E2043
:1001200008006A2005129E2005169E200800223035
:100130009F280E309F207A281B309F281C308F006C
:100140008F0BA0280034A328FF3FFF3FFF3FFF3F56
:10015000FF3FFF3FFF3FFF3FFF3FFF3FFF3FFF3FAF
:10016000FF3FFF3FFF3FFF3FFF3FFF3FFF3FFF3F9F
:10017000FF3FFF3FFF3FFF3FFF3FFF3FFF3FFF3F8F
:10018000FF3FFF3FFF3FFF3FFF3FFF3FFF3FFF3F7F
:02400E00F93F78
:10420000FF00FF00FF00FF00FF00FF00FF00FF00B6
:10421000FF00FF00FF00FF00FF00FF00FF00FF00A6
:10422000FF00FF00FF00FF00FF00FF00FF00FF0096
:10423000FF00FF00FF00FF00FF00FF00FF00FF0086
:10424000FF00FF00FF00FF00FF00FF00FF00FF0076
:10425000FF00FF00FF00FF00FF00FF00FF00FF0066
:10426000FF00FF00FF00FF00FF00FF00FF00FF0056
:10427000FF00FF00FF00FF00FF00FF00FF00FF0046
:00000001FF
